:020000040000FA
:1000000000002A00450060007B009600B100CC0093
:10001000E70002011D01380153016E018901A401AD
:10002000BF01DA01F50110022B02460261027C02D7
:100030009702B202CD02E80203031E033903540300
:100040006F038903A403BF03DA03F50310042B0431
:10005000460461047C049704B204CD04E80403055B
:100060001E05390554056F058A05A505C005DB0584
:10007000F60511062C06470662067D069806B306AD
:10008000CE06E90604071F073A07550770078B07D6
:10009000A607C107DC07F70712082D084808630800
:1000A0007E089908B408CF08EA08050920093B0929
:1000B000560971098C09A709C209DD09F809130A53
:1000C0002D0A480A630A7E0A990AB40ACF0AEA0A84
:1000D000050B200B3B0B560B710B8C0BA70BC20BAC
:1000E000DD0BF80B130C2E0C490C640C7F0C9A0CD6
:1000F000B50CD00CEB0C060D210D3C0D570D720DFF
:00000001FF
